:100000000C9432010C94D1010C94F6010C944E0224
:100010000C944F010C944F010C944F010C944F0120
:100020000C944F010C944F010C944F010C94230F2E
:100030000C94B00D0C944F010C94FC030C944F01E4
:100040000C944F010C944F010C944F010C944F01F0
:100050000C944F01574F626974205344433130363A
:1000600045200000C1814001C0804101C0804100A5
:10007000C1814001C0804100C1814000C181400177
:10008000C0804101C0804100C1814000C181400168
:10009000C0804100C1814001C0804101C080410059
:1000A000C1814001C0804100C1814000C181400147
:1000B000C0804100C1814001C0804101C080410039
:1000C000C1814000C1814001C0804101C080410028
:1000D000C1814001C0804100C1814000C181400117
:1000E000C0804101C0804100C1814000C181400108
:1000F000C0804100C1814001C0804101C0804100F9
:10010000C1814001C1814001C0804101C080C10066
:10011000C1814001C080410041814000C181400156
:10012000C0804100C1814001C0804101C0804100C8
:10013000C1814001C0804100C1814000C1814001B6
:10014000C0804101C0804100C1814000C1814001A7
:10015000C0804100C1814001C0804101C080410098
:10016000C1814000C0C101C30302C2C60607C70562
:10017000C5C404CC0C0DCD0FCFCE0E0ACACB0BC913
:100180000908C8D81819D91BDBDA1A1EDEDF1FDDF3
:100190001D1CDC14D4D515D71716D6D21213D311C3
:1001A000D1D010F03031F133F3F23236F6F737F5C3
:1001B0003534F43CFCFD3DFF3F3EFEFA3A3BFB3953
:1001C000F9F83828E8E929EB2B2AEAEE2E2FEF2D53
:1001D000EDEC2CE42425E527E7E62622E2E323E103
:1001E0002120E0A06061A163A3A26266A6A767A523
:1001F0006564A46CACAD6DAF6F6EAEAA6A6BAB6993
:10020000A9A86878B8B979BB7B7ABABE7E7FBF7D72
:10021000BDBC7CB47475B577B7B67672B2B373B142
:100220007170B05090915193535292965657975582
:100230009594549C5C5D9D5F9F9E5E5A9A9B5B99D2
:10024000595898884849894B8B8A4A4E8E8F4F8DD2
:100250004D4C8C4484854587474686824243834182
:100260008180400011241FBECFE5D4E0DEBFCDBFAA
:1002700010E0A0E6B0E0E8ECF3E202C005900D92D9
:10028000AA38B107D9F713E0AAE8B0E001C01D927F
:10029000A43CB107E1F70E94B2020C94E3110C9464
:1002A00000001ABA8FEF87BB84BB81BB0895089505
:1002B000BB9A84B3836084BBA298AA9A13BE83B707
:1002C000896683BF0895AC019A9934C0F894A898C0
:1002D000A9981CBE83B38074682F772711C0A89596
:1002E00082B390E2892782BB20E030E0E0EAFFE0C1
:1002F000CF010197F1F72F5F3F4F2A3F3105C1F73B
:1003000083B39927807490706817790741F320E0D0
:1003100030E0E0EAFFE0CF010197F1F72F5F3F4FB8
:1003200083E0283E3807B9F7959A789480E293E005
:100330000197F1F780918A0090918B009C01429F78
:10034000C001439F900D529F900D1124181619065D
:1003500084F01CBE80E293E0FC013197F1F7A8988D
:10036000A9980197F1F7A89AA99A80E991E00197D5
:10037000F1F7141615061CF4A89AA99805C04115A2
:10038000510511F0A898A99ACA0157FF04C08827FF
:100390009927841B950B8CBF50938B0040938A0048
:1003A00008951F920F920FB60F9211248F939F936F
:1003B000AF93BF938091AE029091AF02A091B00233
:1003C000B091B1020196A11DB11D8093AE02909330
:1003D000AF02A093B002B093B102BF91AF919F91D1
:1003E0008F910F900FBE0F901F9018951F920F9234
:1003F0000FB60F9211248F939F93AF93BF93809169
:10040000AE029091AF02A091B002B091B1020197FB
:10041000A109B1098093AE029093AF02A093B002FC
:10042000B093B102BF91AF919F918F910F900FBE8A
:100430000F901F9018950F931F938C01B801882778
:1004400077FD8095982F0E94C61017FF06C020E008
:1004500030E040E857E40E94211020E030E04AE715
:1004600055E40E9459110E94A910DC01CB010197AB
:10047000F1F71F910F9108959B01AC01E0EAFFE0B5
:1004800007C0CF010197F1F7215030404040504064
:100490002115310541055105A1F708951F920F92CD
:1004A0000FB60F9211242F933F934F935F936F9347
:1004B0007F938F939F93AF93BF93EF93FF93A895F1
:1004C0008091FD019091FE0101969093FE01809331
:1004D000FD018091AE029091AF02A091B002B09167
:1004E000B1028093170290931802A0931902B0935F
:1004F0001A0278949F9904C081E08093110202C08F
:10050000109211029E9B04C081E08093010202C000
:100510001092010283E192E00E948A0560912F020D
:100520007091300280913102909132020E94D0107D
:100530000E94A910DC01CB010E94630188B780688A
:1005400088BFFF91EF91BF91AF919F918F917F9164
:100550006F915F914F913F912F910F900FBE0F9030
:100560001F9018950F931F93CF93DF9320E030E0F7
:10057000E0EAFFE0CF010197F1F72F5F3F4F81E005
:10058000243F3807B9F7A89588E190E02FE00FB62F
:10059000F894A89581BD0FBE21BD02E310E0929AA8
:1005A000C1E3D0E08A9885B7826085BF8BB780644D
:1005B0008BBF939A8B9885B7886085BF8BB780680F
:1005C0008BBF15BC85B58F6085BD89B7806889BF35
:1005D00087E283BD0E945801DE010E94C011802D78
:1005E0008F3F39F40E941F0880E0DE01082E0E9430
:1005F000CD1192E0ECE4F2E0D801192E0E94C8116E
:10060000E9EEF1E0A4E3B0E0192E0E94C811E7E0A2
:10061000F2E0A6E3B0E0192E0E94C81184E043E3A3
:1006200052E0A8E3B0E0FA01182E0E94C8114C5F16
:100630005F4FACE3B0E0FA01182E0E94C8114C5F86
:100640005F4FA0E4B0E0FA01182E0E94C8114C5F81
:100650005F4FA4E4B0E0FA01182E0E94C8114C5F6D
:100660005F4FA8E4B0E0FA01182E0E94C8114C5F59
:100670005F4FACE4B0E0FA01182E0E94C811EEE022
:10068000F2E0A0E5B0E0192E0E94C811E2E0F2E02D
:10069000A2E5B0E0192E0E94C81110921302109228
:1006A0001402109215021092160210921702109264
:1006B00018021092190210921A0210921B02109244
:1006C0001C0210921D0210921E0210921F02109224
:1006D0002002109221021092220280E090E0A0E01D
:1006E000B0E08093230290932402A0932502B0935C
:1006F000260280932F0290933002A0933102B09390
:1007000032028093270290932802A0932902B0938B
:100710002A0280932B0290932C02A0932D02B09377
:100720002E020E949B0D60E081E00E94ED0381B3E8
:10073000806681BB959A969884B38F7384BB85B38A
:10074000806C85BB1ABA8EEF8BBB60E081E00E94A3
:10075000ED037894109200020E94AD07CC990EC070
:10076000F894A4E6B0E00E94C011802D78948F3FE9
:1007700089F00E94680760E670E008C0CF9B04C063
:10078000CE9B02C0CD9906C064E670E08EE492E094
:100790000E94EE0F1092100220E030E0E0EAFFE04D
:1007A000CF010197F1F72F5F3F4F81E0243F3807DA
:1007B000B9F7A8958EE492E00E9428096FE18EE4D3
:1007C00092E00E94820EF5CF97B1907F97B997B1D2
:1007D0008F70982B97B9369A08953E9A96B19F6C70
:1007E00096B99AB3809598239ABB9BB398239BBBE9
:1007F00080E00E94E40308951F920F920FB60F92BB
:1008000011248F939F9384B195B19093FC018093B1
:10081000FB01369A9F918F910F900FBE0F901F9002
:10082000189508952F923F924F925F926F927F9208
:100830008F929F92AF92BF92CF92DF92EF92FF92F0
:100840000F931F93CF93DF93EC012C813D814E8159
:100850005F81688179818A819B810E9420107B0160
:100860008C016C847D848E849F842AE037ED43E282
:100870005BE36C897D898E899F890E9459115B0198
:100880006C01A4019301C801B7010E9421109B01D2
:10089000AC01C601B5010E94591120E030E040E0F2
:1008A0005FE30E945911288539854A855B850E943E
:1008B00021101B012C01EC86FD860E871F87288DD9
:1008C000398D4A8D5B8DC801B7010E9459115B01BA
:1008D0006C01A4019301C801B7010E94201020E01F
:1008E00030E048EC53E40E9459112C8D3D8D4E8D23
:1008F0005F8D0E9459119B01AC01C601B5010E9498
:100900002110A20191010E9421105B016C01688BF2
:10091000798B8A8B9B8BECA0FDA00EA11FA1A80157
:1009200097010E94EC10181664F0E8A0F9A00AA143
:100930001BA1A8019701C601B5010E94E9108823F7
:100940004CF4E88AF98A0A8B1B8BE886F9860A87B9
:100950001B8704C0288639864A865B86DF91CF9143
:100960001F910F91FF90EF90DF90CF90BF90AF90CD
:100970009F908F907F906F905F904F903F902F90BF
:1009800008954F925F926F927F928F929F92AF9253
:10099000BF92CF92DF92EF92FF920F931F93CF936C
:1009A000DF93CDB7DEB724970FB6F894DEBF0FBE46
:1009B000CDBF6C0149835A836B837C838F8C98A055
:1009C000A9A0BAA04F88588C698C7A8C23ED3DE49D
:1009D00042E95FE3C301B2010E9459117B018C011E
:1009E0002CEB34E743ED5EEB6B8D7C8D8D8D9E8D16
:1009F0000E9459119B01AC01C801B7010E9421104E
:100A00007B018C012AE333E24AE85DE369817A8164
:100A10008B819C810E9459119B01AC01C801B701D7
:100A20000E9421107B018C0129ED35E24AE05EE352
:100A3000C501B4010E9459119B01AC01C801B70165
:100A40000E9421107B018C012AE333E24AE85DE336
:100A50006BA17CA18DA19EA10E9459119B01AC01AB
:100A6000C801B7010E942110F60184869586A686EA
:100A7000B78629813A814B815C8120873187428703
:100A80005387448255826682778260837183828332
:100A90009383C60124960FB6F894DEBF0FBECDBF78
:100AA000DF91CF911F910F91FF90EF90DF90CF904A
:100AB000BF90AF909F908F907F906F905F904F907E
:100AC0000895AF92BF92CF92DF92EF92FF920F9371
:100AD0001F935B016C0179018A010E94EC101816CA
:100AE00074F017FB109517F91095A8019701C6012E
:100AF000B5010E94E91087FD02C086017501C80199
:100B0000B7011F910F91FF90EF90DF90CF90BF90B2
:100B1000AF9008952F923F924F925F926F927F9283
:100B20008F929F92AF92BF92CF92DF92EF92FF92FD
:100B30000F931F93CF93DF93EC01688179818A81B2
:100B40009B812C813D814E815F81621B730B840BE5
:100B5000950B0E94C6101B012C01609394007093AA
:100B6000950080939600909397006C817D818E8193
:100B70009F81288539854A855B85621B730B840BB1
:100B8000950B0E94C6106C8B7D8B8E8B9F8BEC8897
:100B9000FD880E891F89688579858A859B852C85C6
:100BA0003D854E855F85621B730B840B950B0E9400
:100BB000C6109B01AC01C801B7010E9420106093D0
:100BC0009000709391008093920090939300809195
:100BD0000102882309F0B3C080910002813059F4EA
:100BE0006091C2037091C303882777FD8095982F89
:100BF0000E94C6102AC080910002823009F05DC0B8
:100C000068A979A98AA99BA90091FB011091FC010F
:100C100020E030EC4FE754E40E9463106B017C014C
:100C2000B801882777FD8095982F0E94C61017FF7E
:100C300006C020E030E040E857E40E9421109B010C
:100C4000AC01C701B6010E9459119B01AC01609330
:100C50008C0070938D0080938E0090938F00809114
:100C60001102882359F0DA01C901B05880938C0031
:100C700090938D00A0938E00B0938F00A88CB98CB8
:100C8000CA8CDB8CECA8FDA80EA91FA9288D398D74
:100C90004A8D5B8D60918C0070918D0080918E00EB
:100CA00090918F000E942010A80197010E94610579
:100CB0009B01AC01C601B50125C0809100028823CB
:100CC00009F05DC028A139A14AA15BA1688C798C8B
:100CD0008A8C9B8CACA8BDA8CEA8DFA8E88CF98C28
:100CE0000A8D1B8DC201B1010E945911A801970103
:100CF0000E942010A60195010E9461059B01AC0194
:100D0000C401B3010E94211060938C0070938D0088
:100D100080938E0090938F0028A939A94AA95BA9D6
:100D20000E94610560938C0070938D0080938E000B
:100D300090938F00688F798F8A8F9B8F20C080E07F
:100D400090E0A0E0B0E080938C0090938D00A093A1
:100D50008E00B0938F008C8B9D8BAE8BBF8B888F5A
:100D6000998FAA8FBB8F8093900090939100A0934E
:100D70009200B0939300888B998BAA8BBB8B2C89A4
:100D80003D894E895F89ECA0FDA00EA11FA1A8A4FA
:100D9000B9A4CAA4DBA460918C0070918D008091ED
:100DA0008E0090918F000E942010A80197010E9450
:100DB00059112091900030919100409192005091F2
:100DC00093000E942010A60195010E945911609382
:100DD0008C0070938D0080938E0090938F00E88834
:100DE000F9880A891B892AE037ED43E25BE30E9418
:100DF00059119B01AC01C801B7010E9421106C8FF1
:100E00007D8F8E8F9F8F2CA53DA54EA55FA56C8DE8
:100E10007D8D8E8D9F8D0E9461056C8F7D8F8E8F55
:100E20009F8F8C8D9D8DAE8DBF8D888B998BAA8B5E
:100E3000BB8B88859985AA85BB858C879D87AE8766
:100E4000BF878C819D81AE81BF8188879987AA8762
:100E5000BB87DF91CF911F910F91FF90EF90DF90B3
:100E6000CF90BF90AF909F908F907F906F905F904A
:100E70004F903F902F9008950F931F938C01FC018A
:100E8000248135814681578160817181828193817E
:100E90000E942010F80120893189428953890E94DB
:100EA0005911F8016087718782879387248D358D6A
:100EB000468D578D0E946105F80160877187828792
:100EC000938764877587868797871F910F91089509
:100ED00088E10FB6F89481BD11BC0FBEF89424E6EA
:100EE00030E0E2EBF2E0D9010E94C011802D992799
:100EF0008083882339F02F5F3F4F319681E023367E
:100F0000380789F77894A89588E190E02FE00FB62C
:100F1000F894A89581BD0FBE21BD089588E10FB654
:100F2000F89481BD11BC0FBEF89484E690E02FEFD9
:100F3000DC01022E0E94CD11019631E08336930729
:100F4000B9F77894A89588E190E02FE00FB6F8946F
:100F5000A89581BD0FBE21BD089588E10FB6F89414
:100F600081BD11BC0FBEF894E2EBF2E0119283E078
:100F7000E13BF807D9F77894A89588E190E02FE055
:100F80000FB6F894A89581BD0FBE21BD0895F894C1
:100F900092E0ECE4F2E0A2E3B0E0192E0E94DE1150
:100FA000E9EEF1E0A4E3B0E0192E0E94DE11E7E0E3
:100FB000F2E0A6E3B0E0192E0E94DE1184E043E3E4
:100FC00052E0A8E3B0E0FA01182E0E94DE114C5F57
:100FD0005F4FACE3B0E0FA01182E0E94DE114C5FC7
:100FE0005F4FA0E4B0E0FA01182E0E94DE114C5FC2
:100FF0005F4FA4E4B0E0FA01182E0E94DE114C5FAE
:101000005F4FA8E4B0E0FA01182E0E94DE114C5F99
:101010005F4FACE4B0E0FA01182E0E94DE11EEE062
:10102000F2E0A0E5B0E0192E0E94DE11E2E0F2E06D
:10103000A2E5B0E0192E0E94DE117894089586E9A9
:1010400090E090934D0280934C0282E390E0909365
:10105000EA018093E90184E190E090930802809393
:1010600007028FE692E1A3E0BCE380933302909302
:101070003402A0933502B093360280E090E0A0EEF7
:10108000B0E48093370290933802A0933902B09372
:101090003A0280933B0290933C02A0933D02B093AE
:1010A0003E0280E090E0AFE7B3E480933F0290938C
:1010B0004002A0934102B093420280E090E0ADEC88
:1010C000B3E48093430290934402A0934502B0930B
:1010D00046028AE097EDA3E2B0E480934702909342
:1010E0004802A0934902B0934A0280E090E19093B5
:1010F0000F0280930E028AE090E0909303028093A7
:101100000202109213021092140210921502109211
:1011100016021092170210921802109219021092E1
:101120001A0210921B0210921C0210921D021092C1
:101130001E0210921F0210922002109221021092A1
:10114000220280E090E0A0E0B0E080932302909340
:101150002402A0932502B093260280932F0290933D
:101160003002A0933102B093320280932702909311
:101170002802A0932902B0932A0280932B02909315
:101180002C02A0932D02B0932E020E94C70708954F
:10119000CF93DF93C0E0D0E002C00E94EA0DEC2FB5
:1011A000FF27EE54FD4F8081882329F0219691E09E
:1011B000C030D90791F7DF91CF910895CF93DF9396
:1011C00088E10FB6F89481BD11BC0FBEF8940E945F
:1011D0008E0782EB92E0EC0109900020E9F7C81B32
:1011E000D90BA4E6B0E0FC01219724F001900E9405
:1011F000CD11FACF7894A89588E190E02FE00FB652
:10120000F894A89581BD0FBE21BDDF91CF910895BF
:101210000E94AD076AE08EE492E00E94820E68E6CA
:1012200070E08EE492E00E94E50F892B69F06EE495
:1012300072E082EB92E00E94DA0F6CE670E082EBE3
:1012400092E00E94DA0FE6CF8EE20E94EA0D089546
:10125000AF92BF92CF92DF92EF92FF920F931F93C4
:10126000CF93DF93EC018881813209F0FBC2898141
:10127000883509F4F5C28935B0F4813509F4F0C236
:10128000823550F4853409F4E6C2803509F413C27E
:10129000843409F0E7C2DCC2863509F470C18735B1
:1012A00008F0ECC0DFC28A3609F446C18B3650F430
:1012B000823609F402C1853609F425C18A3509F060
:1012C000D1C2B4C28F3609F431C1803720F48D36D3
:1012D00009F0C8C207C0823709F42CC18A3709F067
:1012E000C1C24DC28A818A36A1F08B3620F4813684
:1012F00009F0B8C20AC0803729F0833709F0B2C2BA
:1013000081E004C010920002ADC282E0809300022E
:10131000A9C281E080930002ABC0CF9944C0CE99AE
:1013200042C0CD9940C01092C3031092C2031092E4
:10133000C3031092C20325C06AEF70E080E090E022
:101340000E943C0282B390E4892782BB8091C20351
:101350009091C303892B31F460ED77E080E090E059
:101360000E943C02CF9939C0CE994AC0CD995BC04A
:101370008091C2039091C30301969093C30380931D
:10138000C2030091C2031091C303609143027091A4
:10139000440280914502909146020E94A910601774
:1013A000710754F656C0CF9905C080914C029091B8
:1013B0004D0206C0CE990AC08091E9019091EA01E0
:1013C0009093C3038093C20381E041C0CD993EC096
:1013D0008091070290910802F3CF8091C20390910F
:1013E000C30390934D0280934C02F89482E0ECE4A6
:1013F000F2E0A2E3B0E0182E0E94DE11789429C03A
:101400008091C2039091C3039093EA018093E90114
:10141000F89482E0E9EEF1E0A4E3B0E0182E0E9437
:10142000DE11789416C08091C2039091C30390930B
:10143000080280930702F89482E0E7E0F2E0A6E376
:10144000B0E0182E0E94DE11789403C082E08093F1
:1014500000028091980090919900019690939900D4
:1014600080939800892B21F482B390E4892782BB72
:101470000E94FC0D882309F450CFF4C1CE010296DE
:101480000E948E0F20E931E0A901849F9001859F81
:10149000300D949F300D112430939B0020939A00BF
:1014A0001092FE011092FD018091FD019091FE01CC
:1014B0008217930708F0D6C1F7CF8A818037A9F049
:1014C000813730F48536B9F08C3609F0CBC110C0C5
:1014D000833741F08437A1F0823709F0C3C10E94FD
:1014E0000809C0C10E94DE08BDC10E94EF0CBAC14C
:1014F0000E946807B7C10E948E070E94AD07B2C163
:101500000E94C808AFC162E08EE092E00E94FD0E2A
:1015100080910E0290910F02892B09F0A3C181E006
:1015200090E090930F0280930E029CC162E082E0F3
:1015300092E0D7C0F894FFCF8A81893771F08A375B
:10154000A9F0883709F08EC1CE0103960E948E0F54
:1015500090934D0280934C0285C1CE0103960E9468
:101560008E0F9093EA018093E9017CC1CE0103962E
:101570000E948E0F909308028093070273C180919E
:101580000002813069F5E0900E02F0900F02CE016A
:1015900002960E948E0FAA2797FDA095BA2FBC0134
:1015A000CD010E94C6102AE037ED43E25BE30E94C2
:1015B00059115B016C010027F7FC0095102FC80141
:1015C000B7010E94C6109B01AC01C601B5010E9483
:1015D00059110E94A9107093C3036093C20342C1C2
:1015E00080910002882309F03DC1E0900E02F09046
:1015F0000F02CE0102960E94AC0F0027F7FC009567
:10160000102FA80197010E94A111609313027093FB
:101610001402809315029093160282B390E48927F6
:1016200082BBE0901702F09018020091190210910D
:101630001A02209113023091140240911502509128
:1016400016028091020290910302AA2797FDA095AD
:10165000BA2F281B390B4A0B5B0B2E153F05400791
:10166000510714F5E0901702F0901802009119024A
:1016700010911A0220911302309114024091150228
:10168000509116028091020290910302AA2797FDC1
:10169000A095BA2F280F391F4A1F5B1FE216F306C9
:1016A000040715070CF4DEC064E170E080E090E010
:1016B0000E943C02B2CF8A81873569F1883530F4C7
:1016C0008534C1F1853509F0CDC016C0843731F0BD
:1016D000873751F0853609F0C5C00AC064E083E35E
:1016E00092E00E94FD0EBEC064E087E392E0F9CF75
:1016F00064E08BE392E0F5CFCE0103960E94AC0F3D
:101700000E94C61060933F02709340028093410292
:1017100090934202A7C0CE0103960E94AC0F0E9494
:10172000C6106093430270934402809345029093E5
:10173000460298C0CE0103960E94AC0F0E94C610CC
:1017400060934702709348028093490290934A0243
:1017500060914702709148028091490290914A023B
:1017600020E030E04AE754E40E94631060934702AF
:10177000709348028093490290934A0273C0F89490
:101780001092AE021092AF021092B0021092B1020B
:101790001092130210921402109215021092160267
:1017A0001092130210921402109215021092160257
:1017B00010921702109218021092190210921A0237
:1017C00010921B0210921C0210921D0210921E0217
:1017D00010921F02109220021092210210922202F7
:1017E00080E090E0A0E0B0E0809323029093240298
:1017F000A0932502B093260280932F02909330028B
:10180000A0933102B0933202809327029093280272
:10181000A0932902B0932A0280932B0290932C026A
:10182000A0932D02B0932E0278941CC06EE670E057
:10183000CE0102960E94E50F892BA1F4F89480E076
:1018400090E0AEEFB1E00C010E94D91178940AC08B
:101850000E941F0807C01092C3031092C20302C067
:101860000E94C70788818F3309F0ADC08981853612
:1018700021F1863648F4803509F44AC0863529F1CD
:10188000893409F0A0C098C08F36D9F0863721F08E
:101890008A3609F098C07DC08A81803721F083376D
:1018A00009F091C004C064E087E192E003C064E005
:1018B00087E292E00E94E50E86C062E08EE092E050
:1018C000F9CF62E082E092E0F5CF8A81803721F0A3
:1018D000833709F078C004C064E083E192E0EACF86
:1018E00080911102882341F08091C2039091C3033B
:1018F000909581959F4F04C08091C2039091C3033E
:101900009093A1008093A00062E080EA90E0D2CFA3
:101910008A81873501F1883530F4853401F18535C8
:1019200009F051C014C0843731F0873741F0853653
:1019300009F049C008C064E083E392E0BBCF64E0F3
:1019400087E392E0B7CF64E08BE392E0B3CF64E04B
:101950008FE392E0AFCF64E083E492E0ABCF60919D
:101960004702709148028091490290914A0220E01A
:1019700030E04AE754E40E94591160939C00709350
:101980009D0080939E0090939F0064E08CE990E01E
:1019900091CF8A81893741F08A3751F0883799F49D
:1019A00062E08CE492E086CF62E089EE91E082CF43
:1019B00062E087E092E07ECF86E790E00E945F0ED3
:1019C0008DE00E94EA0D9698DF91CF911F910F91C3
:1019D000FF90EF90DF90CF90BF90AF9008950F935E
:1019E0001F93EEE6F2E0119282E0E03AF807D9F7B1
:1019F00000E040E020E030E0E2EBF2E0DF010D90BB
:101A00000020E9F71197AE1BBF0B0FC0EE54FD4F3E
:101A100080818D3041F4E02FFF27E259FD4F408354
:101A20000F5F492F4F5F2F5F3F4F922FE22FFF270E
:101A3000EA17FB0758F310E078C08091B2038132B7
:101A4000B1F58091B3038A3419F0833581F505C06F
:101A500084EB93E00E948E0F29C08091B4038233FF
:101A600089F0833318F4813311F505C0833389F08D
:101A70008433E9F415C0C9991AC085EB93E00E943C
:101A80008E0F14C0CA9913C085EB93E00E948E0F8D
:101A90000DC0CB990CC085EB93E00E948E0F06C061
:101AA000CC9905C085EB93E00E948E0F182FE12F93
:101AB000FF27E259FD4F608140E050E08181282FEF
:101AC00033272150304006C0EE54FC4FAE54BD4F7A
:101AD0008C918083942F862F840F4F5F5F4FA82FA8
:101AE000BB27E92FFF27A217B30774F3EE54FC4F6F
:101AF00010820E94FC0D882399F06AE08EE492E047
:101B00000E94820E42E050E067E870E08EE492E0CE
:101B10000E94F50F892B61F00E94450E0E944D0E28
:101B200082EB93E00E9428091F5F101708F485CF0D
:101B30001F910F91089580E189B988E98AB986E8F3
:101B400080BD1092B1031092AD0210920902109262
:101B5000FF011092AA0208958AB187708AB9089588
:101B60001F920F920FB60F9211248F939F93EF93B2
:101B7000FF939091FF0180910902981781F0E09105
:101B80000902EF5FEF73E093A300E0930902FF27E0
:101B9000EA55FE4F80818093A2008CB901C0559810
:101BA000FF91EF919F918F910F900FBE0F901F901B
:101BB00018959091AD028091B1039817D1F3E091FF
:101BC000B103EF5FE093B103FF27EA55FF4F808138
:101BD00099270895282F9091FF019F5F9F7380910F
:101BE00009029817E1F3E92FFF27EA55FE4F2083FA
:101BF0009093FF01559A08959091AD028091B103A1
:101C000020E030E0981711F021E030E0C90108959C
:101C10009091FF018091090220E030E0981711F0C7
:101C200021E030E0C90108952FB7F8949091AD02FA
:101C30008091B103981740F08091AD029091B1036B
:101C40002FBF891B992708958091AD029091B10310
:101C50002FBF891B992708952FB7F8949091FF0102
:101C600080910902981740F08091FF01909109023C
:101C70002FBF891B992708958091FF019091090238
:101C80002FBF891B805C992708958FB7F894109215
:101C9000FF01109209028FBF08958FB7F894109238
:101CA000AD021092B1038FBF089580E00E94EA0D4B
:101CB0008DE00E94EA0D8AE00E94EA0D0895CF921D
:101CC000DF92EF92FF920F931F93CF93DF936C01FC
:101CD000C0E0D0E0EC2EFF2486010E0D1F1DF801A0
:101CE00080810E94EA0D2196F8018081882391F776
:101CF000C701DF91CF911F910F91FF90EF90DF907F
:101D0000CF900895EF92FF920F931F93CF93DF939D
:101D1000EC01062F10E014C07E01E80EF91E0E94AF
:101D2000D90DF70180838D3021F08A3011F088239E
:101D300031F4F70110821F5F812F992709C01F5FBF
:101D4000812F9927101741F7C80FD91F21971882A3
:101D5000DF91CF911F910F91FF90EF900895982FF1
:101D6000E091AD02EF5FE093AD028091B103E8171F
:101D700041F48FB7F8941092AD021092B1038FBF67
:101D80000895FF27EA55FF4F90830895EF92FF9241
:101D90000F931F93CF93DF937C01C0E0D0E002C08C
:101DA0000E94AF0E0C2F1127F701E00FF11F808169
:101DB00021968823A9F70E94AF0EC801DF91CF9129
:101DC0001F910F91FF90EF900895FF920F931F9333
:101DD000CF93DF938C01F62EEC0103C089910E9412
:101DE000EA0DC8018F0D911DC817D907B9F7DF910A
:101DF000CF911F910F91FF900895FF920F931F9322
:101E0000CF93DF938C01F62EEC0103C00E94D90D15
:101E10008993C8018F0D911DC817D907B9F7DF91B4
:101E2000CF911F910F91FF9008950F931F930EE490
:101E300012E0BC01C8010E94D30FC8010E945F0ECE
:101E40001F910F9108951F920F920FB60F921124B8
:101E50002F933F934F935F936F937F938F939F93B2
:101E6000AF93BF93EF93FF939CB19093A500E09144
:101E7000AD02EF5FE093A400E093AD028091B10367
:101E8000E81741F48FB7F8941092AD021092B103A5
:101E90008FBF04C0FF27EA55FF4F90838091100247
:101EA000882319F0892F0E94EA0DFF91EF91BF91CD
:101EB000AF919F918F917F916F915F914F913F91E2
:101EC0002F910F900FBE0F901F901895DC018FEF90
:101ED0008093E7018093E6014091E8012FEF5FEFE7
:101EE0000DC04D914527842F9927FC01ED59FF4FD7
:101EF000549152278D599E4FFC012491615088F7CF
:101F00002093E6014093E8015093E701852F99273C
:101F1000982F88273327822B932B0895FC0188273D
:101F20009927E89421912032E9F3293010F02E30DE
:101F3000C8F32B3241F02D3239F4689404C00E946A
:101F40001810820F911D219120532A30C0F31EF4E6
:101F5000909581959F4F08951F93FC01992788279D
:101F6000BC01E89411911032E9F3193010F01E30E1
:101F7000C8F31B3251F01D3249F4689406C00E9428
:101F80000310610F711D811D911D119110531A30A5
:101F9000B0F33EF490958095709561957F4F8F4F8B
:101FA0009F4F1F910895FB01DC0105900D920020C9
:101FB000E1F70895FB01DC010D900020E9F711978E
:101FC00001900D920020E1F70895FB01DC018D9155
:101FD000019080190110D9F3990B0895FB01DC01E0
:101FE00001900D920020E1F70895FB01DC014150C2
:101FF000504030F08D910190801919F40020B9F70C
:10200000881B990B0895592F482F372F262F660FBD
:10201000771F881F991F660F771F881F991F620FF0
:10202000731F841F951F660F771F881F991F0895C0
:102030007AE0979F902D879F802D910D1124089510
:102040005058192E08D101D0EBC0BA176207730798
:1020500084079507B1F188F40EF410940B2EBA2F73
:10206000A02D062E622F202D072E732F302D082E27
:10207000842F402D092E952F502DFF275523B9F081
:10208000591B49F0573E98F0469537952795A795E7
:10209000F0405395C9F776F0BA0F621F731F841F83
:1020A00030F4879577956795B795F040939517FA33
:1020B0000F2E0895BF1BBB27BA0B620B730B840B4B
:1020C000F6CFDEF6F4C0C7D001D0AAC0552359F030
:1020D000992369F09F575F57951B33F442F490386A
:1020E00011F4915805C0B4C091589F3F09F4DFC066
:1020F000BB27112462177307840730F4660F771F1C
:10210000881FBB1F915098F311D00F920FD00F92E0
:102110000DD0A0E82617370748071B0609F0A0488E
:10212000BA2F602D7F918F9100240895A0E800249C
:10213000621773078407B10528F0621B730B840BC9
:10214000B1090A2A660F771F881FBB1FA69581F762
:10215000089597FB8CD09F3738F0FEE9F91B982F34
:10216000872F762F6B2F05C09FC096958795779503
:102170006795F150D0F73EF49095809570956195F4
:102180007F4F8F4F9F4F0895E89403C097FB0EF445
:10219000F3DFB62F672F782F892F9EE9002440C0E8
:1021A00074D09F3760F40EF07FC09FEB80E87727F4
:1021B00066270895869577956795B11D939596390D
:1021C000C8F32EF4BB2319F06F5F7F4F8F4FBB27EF
:1021D00027C00ED05EF004C00BD026F001C008D09E
:1021E00019F020F48FEF089580E0089581E00895BC
:1021F00097FB092E052600F8689430D0E89407FC78
:1022000007C0621773078407950721F008F400944C
:102210000794989408959A95BB0F661F771F881F9F
:1022200011249923A1F08823B2F79F3F59F0BB0FE7
:1022300048F421F4002011F460FF04C06F5F7F4F69
:102240008F4F9F4F881F9795879597F908952CC0BA
:102250009FEF80EC0895052E092607FA440F551FBD
:102260005F3F79F0AA27A51708F051E04795880F3E
:10227000991F9F3F31F0BB27B91708F091E0879570
:1022800008959F919F911124E3CF97FB880F991F89
:102290009F3F31F0BB27B91708F091E0879508956B
:1022A0009F919F911124D4CF66277727882799275C
:1022B0000895D1DF01D0B4CF992339F0552329F007
:1022C0009F575F57950F13F49AF1F1CF91589F3FA5
:1022D000E1F3629FA12D0F92BB27639FA00DB11D5B
:1022E000EE27729FA00DB11DEE1FAF93AA27649F2A
:1022F000B00DE11D739FB00DE11DAA1F6627829FDF
:10230000B00DE11DA61F5527749FE00DA11D551F9F
:10231000839FE00DA11D561F849FA00D511D852F89
:102320007A2F6E2F1F900F9088231AF4939539F40B
:102330008FCF000C111CBB1F661F771F881F012841
:102340000895629FD001739FF001829FE00DF11DFF
:10235000649FE00DF11D929FF00D839FF00D749F1F
:10236000F00D659FF00D9927729FB00DE11DF91FCB
:10237000639FB00DE11DF91FBD01CF011124089528
:10238000E199FECFBFBBAEBBE09A11960DB20895A6
:10239000F7DF01921A94E1F70895E199FECFBFBBF0
:1023A000AEBB0DBA11960FB6F894E29AE19A0FBE41
:1023B0000895F3DF012CF1DF112408950190EDDF82
:0823C0001A94E1F70895FFCF24
:1023C80021627000216D6A00216273000D0076653C
:1023D8007273696F6E005344433130364520766519
:0A23E800722E20322E330021450032
:00000001FF
